:020000040000FA
:1000000028046804A304C305000A0008AB04040024
:10001000E707070A0400E7060A0AC10C21000400EA
:10002000010243070F0A250C2100040001024307C7
:10003000150AE706AB05A305450A0C05050C2E00BD
:100040000009CA06200A0400E707230A0400E7069D
:10005000260A04004607300AE707290AA3050F0A03
:10006000F80C6C01AA050A0C380000093802430795
:10007000350AA305410AFF0FFF0FFF0FFF0FFF0F08
:100080000000000000000000000000000000000070
:100090000000000000000000000000000000000060
:1000A0000000000000000000000000000000000050
:1000B0000000000000000000000000000000000040
:020000040000FA
:02100000FF0FE0
:020000040000FA
:02100200FF0FDE
:020000040000FA
:02100400FF0FDC
:020000040000FA
:02100600FF0FDA
:020000040000FA
:021FFE000500DC
:00000001FF
